Component: ARM Compiler 5.06 update 5 (build 528) Tool: armlink [4d35e2]

==============================================================================

Section Cross References

    event_groups.o(.text) refers to heap_1.o(.text) for pvPortMalloc
    event_groups.o(.text) refers to list.o(.text) for vListInitialise
    event_groups.o(.text) refers to tasks.o(.text) for vTaskSuspendAll
    event_groups.o(.text) refers to port.o(.text) for vPortEnterCritical
    queue.o(.text) refers to port.o(.text) for vPortEnterCritical
    queue.o(.text) refers to tasks.o(.text) for xTaskRemoveFromEventList
    queue.o(.text) refers to list.o(.text) for vListInitialise
    queue.o(.text) refers to heap_1.o(.text) for pvPortMalloc
    queue.o(.text) refers to memcpya.o(.text) for __aeabi_memcpy
    tasks.o(.text) refers to list.o(.text) for vListInitialise
    tasks.o(.text) refers to port.o(.text) for vPortEnterCritical
    tasks.o(.text) refers to memseta.o(.text) for __aeabi_memset
    tasks.o(.text) refers to heap_1.o(.text) for pvPortMalloc
    tasks.o(.text) refers to tasks.o(.bss) for pxReadyTasksLists
    tasks.o(.text) refers to tasks.o(.data) for pxDelayedTaskList
    tasks.o(.text) refers to main.o(.text) for vApplicationIdleHook
    tasks.o(.text) refers to main.o(.bss) for ulTaskNumber
    heap_1.o(.text) refers to tasks.o(.text) for vTaskSuspendAll
==============================================================================

Removing Unused input sections from the image.

    Removing event_groups.o(.text), (724 bytes).
    Removing queue.o(.text), (1716 bytes).
    Removing startup_mps_cm3.o(HEAP), (0 bytes).
    Removing dadd.o(.text), (334 bytes).
    Removing dmul.o(.text), (228 bytes).
    Removing ddiv.o(.text), (222 bytes).
    Removing dfixul.o(.text), (48 bytes).
    Removing cdrcmple.o(.text), (48 bytes).
    Removing depilogue.o(.text), (186 bytes).

9 unused section(s) (total 3506 bytes) removed from the image.

==============================================================================

Image Symbol Table

    Local Symbols

    Symbol Name                              Value     Ov Type        Size  Object(Section)

    RESET                                    0x00000000   Section      192  startup_mps_cm3.o(RESET)
    ../clib/microlib/division.c              0x00000000   Number         0  uldiv.o ABSOLUTE
    ../clib/microlib/division.c              0x00000000   Number         0  uidiv.o ABSOLUTE
    ../clib/microlib/init/entry.s            0x00000000   Number         0  entry7a.o ABSOLUTE
    ../clib/microlib/init/entry.s            0x00000000   Number         0  entry11b.o ABSOLUTE
    ../clib/microlib/init/entry.s            0x00000000   Number         0  entry11a.o ABSOLUTE
    ../clib/microlib/init/entry.s            0x00000000   Number         0  entry10b.o ABSOLUTE
    ../clib/microlib/init/entry.s            0x00000000   Number         0  entry8a.o ABSOLUTE
    ../clib/microlib/init/entry.s            0x00000000   Number         0  entry10a.o ABSOLUTE
    ../clib/microlib/init/entry.s            0x00000000   Number         0  entry9b.o ABSOLUTE
    ../clib/microlib/init/entry.s            0x00000000   Number         0  entry9a.o ABSOLUTE
    ../clib/microlib/init/entry.s            0x00000000   Number         0  entry7b.o ABSOLUTE
    ../clib/microlib/init/entry.s            0x00000000   Number         0  entry8b.o ABSOLUTE
    ../clib/microlib/init/entry.s            0x00000000   Number         0  entry.o ABSOLUTE
    ../clib/microlib/init/entry.s            0x00000000   Number         0  entry2.o ABSOLUTE
    ../clib/microlib/init/entry.s            0x00000000   Number         0  entry5.o ABSOLUTE
    ../clib/microlib/longlong.c              0x00000000   Number         0  llsshr.o ABSOLUTE
    ../clib/microlib/longlong.c              0x00000000   Number         0  llushr.o ABSOLUTE
    ../clib/microlib/longlong.c              0x00000000   Number         0  llshl.o ABSOLUTE
    ../clib/microlib/printf/printf.c         0x00000000   Number         0  printf0.o ABSOLUTE
    ../clib/microlib/printf/printf.c         0x00000000   Number         0  printfa.o ABSOLUTE
    ../clib/microlib/printf/printf.c         0x00000000   Number         0  printf8.o ABSOLUTE
    ../clib/microlib/printf/printf.c         0x00000000   Number         0  printf7.o ABSOLUTE
    ../clib/microlib/printf/printf.c         0x00000000   Number         0  printf6.o ABSOLUTE
    ../clib/microlib/printf/printf.c         0x00000000   Number         0  printf5.o ABSOLUTE
    ../clib/microlib/printf/printf.c         0x00000000   Number         0  printf3.o ABSOLUTE
    ../clib/microlib/printf/printf.c         0x00000000   Number         0  printf2.o ABSOLUTE
    ../clib/microlib/printf/printf.c         0x00000000   Number         0  printf1.o ABSOLUTE
    ../clib/microlib/printf/printf.c         0x00000000   Number         0  printfb.o ABSOLUTE
    ../clib/microlib/printf/printf.c         0x00000000   Number         0  printf4.o ABSOLUTE
    ../clib/microlib/printf/stubs.s          0x00000000   Number         0  stubs.o ABSOLUTE
    ../clib/microlib/stdio/streams.c         0x00000000   Number         0  stdout.o ABSOLUTE
    ../clib/microlib/string/memcpy.c         0x00000000   Number         0  memcpyb.o ABSOLUTE
    ../clib/microlib/string/memcpy.c         0x00000000   Number         0  memcpya.o ABSOLUTE
    ../clib/microlib/string/memset.c         0x00000000   Number         0  memseta.o ABSOLUTE
    ../clib/microlib/stubs.s                 0x00000000   Number         0  iusefp.o ABSOLUTE
    ../fplib/microlib/fpadd.c                0x00000000   Number         0  dadd.o ABSOLUTE
    ../fplib/microlib/fpdiv.c                0x00000000   Number         0  ddiv.o ABSOLUTE
    ../fplib/microlib/fpepilogue.c           0x00000000   Number         0  depilogue.o ABSOLUTE
    ../fplib/microlib/fpfix.c                0x00000000   Number         0  dfixul.o ABSOLUTE
    ../fplib/microlib/fpmul.c                0x00000000   Number         0  dmul.o ABSOLUTE
    ..\..\FreeRTOS\croutine.c                0x00000000   Number         0  croutine.o ABSOLUTE
    ..\..\FreeRTOS\event_groups.c            0x00000000   Number         0  event_groups.o ABSOLUTE
    ..\..\FreeRTOS\list.c                    0x00000000   Number         0  list.o ABSOLUTE
    ..\..\FreeRTOS\portable\MemMang\heap_1.c 0x00000000   Number         0  heap_1.o ABSOLUTE
    ..\..\FreeRTOS\portable\RVDS\ARM_CM3\port.c 0x00000000   Number         0  port.o ABSOLUTE
    ..\..\FreeRTOS\queue.c                   0x00000000   Number         0  queue.o ABSOLUTE
    ..\..\FreeRTOS\tasks.c                   0x00000000   Number         0  tasks.o ABSOLUTE
    ..\..\FreeRTOS\timers.c                  0x00000000   Number         0  timers.o ABSOLUTE
    ..\\..\\FreeRTOS\\portable\\RVDS\\ARM_CM3\\port.c 0x00000000   Number         0  port.o ABSOLUTE
    ..\common\basic_io.c                     0x00000000   Number         0  basic_io.o ABSOLUTE
    cdrcmple.s                               0x00000000   Number         0  cdrcmple.o ABSOLUTE
    dc.s                                     0x00000000   Number         0  dc.o ABSOLUTE
    handlers.s                               0x00000000   Number         0  handlers.o ABSOLUTE
    init.s                                   0x00000000   Number         0  init.o ABSOLUTE
    main.c                                   0x00000000   Number         0  main.o ABSOLUTE
    startup_MPS_CM3.s                        0x00000000   Number         0  startup_mps_cm3.o ABSOLUTE
    .ARM.Collect$$$$00000000                 0x000000c0   Section        0  entry.o(.ARM.Collect$$$$00000000)
    .ARM.Collect$$$$00000001                 0x000000c0   Section        4  entry2.o(.ARM.Collect$$$$00000001)
    .ARM.Collect$$$$00000004                 0x000000c4   Section        4  entry5.o(.ARM.Collect$$$$00000004)
    .ARM.Collect$$$$00000008                 0x000000c8   Section        0  entry7b.o(.ARM.Collect$$$$00000008)
    .ARM.Collect$$$$0000000A                 0x000000c8   Section        0  entry8b.o(.ARM.Collect$$$$0000000A)
    .ARM.Collect$$$$0000000B                 0x000000c8   Section        8  entry9a.o(.ARM.Collect$$$$0000000B)
    .ARM.Collect$$$$0000000D                 0x000000d0   Section        0  entry10a.o(.ARM.Collect$$$$0000000D)
    .ARM.Collect$$$$0000000F                 0x000000d0   Section        0  entry11a.o(.ARM.Collect$$$$0000000F)
    .ARM.Collect$$$$00002712                 0x000000d0   Section        4  entry2.o(.ARM.Collect$$$$00002712)
    __lit__00000000                          0x000000d0   Data           4  entry2.o(.ARM.Collect$$$$00002712)
    .emb_text                                0x000000d4   Section      150  port.o(.emb_text)
    .text                                    0x0000016a   Section        0  list.o(.text)
    .text                                    0x00000200   Section        0  tasks.o(.text)
    prvInitialiseTaskLists                   0x00000201   Thumb Code    64  tasks.o(.text)
    prvAddNewTaskToReadyList                 0x00000241   Thumb Code   156  tasks.o(.text)
    prvInitialiseNewTask                     0x000002dd   Thumb Code   142  tasks.o(.text)
    prvResetNextTaskUnblockTime              0x000003cb   Thumb Code    42  tasks.o(.text)
    prvAddCurrentTaskToDelayedList           0x000005a7   Thumb Code   202  tasks.o(.text)
    prvTaskIsTaskSuspended                   0x00000837   Thumb Code    56  tasks.o(.text)
    prvCheckTasksWaitingTermination          0x00000959   Thumb Code     2  tasks.o(.text)
    prvIdleTask                              0x0000095b   Thumb Code    12  tasks.o(.text)
    prvTaskCheckFreeStackSpace               0x000009f7   Thumb Code    22  tasks.o(.text)
    prvListTasksWithinSingleList             0x00000acb   Thumb Code   106  tasks.o(.text)
    .text                                    0x0000110c   Section        0  heap_1.o(.text)
    .text                                    0x00001190   Section        0  port.o(.text)
    prvTaskExitError                         0x00001191   Thumb Code    22  port.o(.text)
    .text                                    0x00001278   Section        0  main.o(.text)
    .text                                    0x000012fc   Section        0  basic_io.o(.text)
    .text                                    0x00001354   Section       28  startup_mps_cm3.o(.text)
    .text                                    0x00001370   Section        0  memseta.o(.text)
    .text                                    0x00001394   Section        0  uidiv.o(.text)
    .text                                    0x000013c0   Section       36  init.o(.text)
    i.__0printf$3                            0x000013e4   Section        0  printf3.o(i.__0printf$3)
    i.__scatterload_copy                     0x00001404   Section       14  handlers.o(i.__scatterload_copy)
    i.__scatterload_null                     0x00001412   Section        2  handlers.o(i.__scatterload_null)
    i.__scatterload_zeroinit                 0x00001414   Section       14  handlers.o(i.__scatterload_zeroinit)
    i._printf_core                           0x00001424   Section        0  printf3.o(i._printf_core)
    _printf_core                             0x00001425   Thumb Code   436  printf3.o(i._printf_core)
    .conststring                             0x000015dc   Section       39  main.o(.conststring)
    .data                                    0x10000000   Section       56  tasks.o(.data)
    pxDelayedTaskList                        0x10000004   Data           4  tasks.o(.data)
    pxOverflowDelayedTaskList                0x10000008   Data           4  tasks.o(.data)
    uxCurrentNumberOfTasks                   0x1000000c   Data           4  tasks.o(.data)
    xTickCount                               0x10000010   Data           4  tasks.o(.data)
    uxTopReadyPriority                       0x10000014   Data           4  tasks.o(.data)
    xSchedulerRunning                        0x10000018   Data           4  tasks.o(.data)
    uxPendedTicks                            0x1000001c   Data           4  tasks.o(.data)
    xYieldPending                            0x10000020   Data           4  tasks.o(.data)
    xNumOfOverflows                          0x10000024   Data           4  tasks.o(.data)
    uxTaskNumber                             0x10000028   Data           4  tasks.o(.data)
    xNextTaskUnblockTime                     0x1000002c   Data           4  tasks.o(.data)
    xIdleTaskHandle                          0x10000030   Data           4  tasks.o(.data)
    uxSchedulerSuspended                     0x10000034   Data           4  tasks.o(.data)
    .data                                    0x10000038   Section        8  heap_1.o(.data)
    xNextFreeByte                            0x10000038   Data           4  heap_1.o(.data)
    pucAlignedHeap                           0x1000003c   Data           4  heap_1.o(.data)
    .data                                    0x10000040   Section        4  port.o(.data)
    uxCriticalNesting                        0x10000040   Data           4  port.o(.data)
    .data                                    0x10000044   Section       12  main.o(.data)
    .data                                    0x10000050   Section        4  stdout.o(.data)
    .bss                                     0x10000054   Section      180  tasks.o(.bss)
    pxReadyTasksLists                        0x10000054   Data         100  tasks.o(.bss)
    xDelayedTaskList1                        0x100000b8   Data          20  tasks.o(.bss)
    xDelayedTaskList2                        0x100000cc   Data          20  tasks.o(.bss)
    xPendingReadyList                        0x100000e0   Data          20  tasks.o(.bss)
    xSuspendedTaskList                       0x100000f4   Data          20  tasks.o(.bss)
    .bss                                     0x10000108   Section     4096  heap_1.o(.bss)
    ucHeap                                   0x10000108   Data        4096  heap_1.o(.bss)
    .bss                                     0x10001108   Section       12  main.o(.bss)
    STACK                                    0x10001118   Section      512  startup_mps_cm3.o(STACK)

    Global Symbols

    Symbol Name                              Value     Ov Type        Size  Object(Section)

    BuildAttributes$$THM_ISAv4$P$D$K$B$S$PE$A:L22UL41UL21$X:L11$S22US41US21$IEEE1$IW$USESV6$~STKCKD$USESV7$~SHL$OSPACE$ROPI$EBA8$MICROLIB$REQ8$PRES8$EABIv2 0x00000000   Number         0  anon$$obj.o ABSOLUTE
    __ARM_use_no_argv                        0x00000000   Number         0  main.o ABSOLUTE
    __Vectors                                0x00000000   Data           4  startup_mps_cm3.o(RESET)
    _printf_a                                0x00000000   Number         0  stubs.o ABSOLUTE
    _printf_c                                0x00000000   Number         0  stubs.o ABSOLUTE
    _printf_charcount                        0x00000000   Number         0  stubs.o ABSOLUTE
    _printf_d                                0x00000000   Number         0  stubs.o ABSOLUTE
    _printf_e                                0x00000000   Number         0  stubs.o ABSOLUTE
    _printf_f                                0x00000000   Number         0  stubs.o ABSOLUTE
    _printf_flags                            0x00000000   Number         0  stubs.o ABSOLUTE
    _printf_fp_dec                           0x00000000   Number         0  stubs.o ABSOLUTE
    _printf_fp_hex                           0x00000000   Number         0  stubs.o ABSOLUTE
    _printf_g                                0x00000000   Number         0  stubs.o ABSOLUTE
    _printf_i                                0x00000000   Number         0  stubs.o ABSOLUTE
    _printf_int_dec                          0x00000000   Number         0  stubs.o ABSOLUTE
    _printf_l                                0x00000000   Number         0  stubs.o ABSOLUTE
    _printf_lc                               0x00000000   Number         0  stubs.o ABSOLUTE
    _printf_ll                               0x00000000   Number         0  stubs.o ABSOLUTE
    _printf_lld                              0x00000000   Number         0  stubs.o ABSOLUTE
    _printf_lli                              0x00000000   Number         0  stubs.o ABSOLUTE
    _printf_llo                              0x00000000   Number         0  stubs.o ABSOLUTE
    _printf_llu                              0x00000000   Number         0  stubs.o ABSOLUTE
    _printf_llx                              0x00000000   Number         0  stubs.o ABSOLUTE
    _printf_longlong_dec                     0x00000000   Number         0  stubs.o ABSOLUTE
    _printf_longlong_hex                     0x00000000   Number         0  stubs.o ABSOLUTE
    _printf_longlong_oct                     0x00000000   Number         0  stubs.o ABSOLUTE
    _printf_ls                               0x00000000   Number         0  stubs.o ABSOLUTE
    _printf_mbtowc                           0x00000000   Number         0  stubs.o ABSOLUTE
    _printf_n                                0x00000000   Number         0  stubs.o ABSOLUTE
    _printf_o                                0x00000000   Number         0  stubs.o ABSOLUTE
    _printf_p                                0x00000000   Number         0  stubs.o ABSOLUTE
    _printf_percent                          0x00000000   Number         0  stubs.o ABSOLUTE
    _printf_pre_padding                      0x00000000   Number         0  stubs.o ABSOLUTE
    _printf_return_value                     0x00000000   Number         0  stubs.o ABSOLUTE
    _printf_s                                0x00000000   Number         0  stubs.o ABSOLUTE
    _printf_sizespec                         0x00000000   Number         0  stubs.o ABSOLUTE
    _printf_str                              0x00000000   Number         0  stubs.o ABSOLUTE
    _printf_truncate_signed                  0x00000000   Number         0  stubs.o ABSOLUTE
    _printf_truncate_unsigned                0x00000000   Number         0  stubs.o ABSOLUTE
    _printf_u                                0x00000000   Number         0  stubs.o ABSOLUTE
    _printf_wc                               0x00000000   Number         0  stubs.o ABSOLUTE
    _printf_wctomb                           0x00000000   Number         0  stubs.o ABSOLUTE
    _printf_widthprec                        0x00000000   Number         0  stubs.o ABSOLUTE
    _printf_x                                0x00000000   Number         0  stubs.o ABSOLUTE
    __cpp_initialize__aeabi_                  - Undefined Weak Reference
    __cxa_finalize                            - Undefined Weak Reference
    __decompress                              - Undefined Weak Reference
    _clock_init                               - Undefined Weak Reference
    _microlib_exit                            - Undefined Weak Reference
    __main                                   0x000000c1   Thumb Code     0  entry.o(.ARM.Collect$$$$00000000)
    _main_stk                                0x000000c1   Thumb Code     0  entry2.o(.ARM.Collect$$$$00000001)
    _main_scatterload                        0x000000c5   Thumb Code     0  entry5.o(.ARM.Collect$$$$00000004)
    __main_after_scatterload                 0x000000c9   Thumb Code     0  entry5.o(.ARM.Collect$$$$00000004)
    _main_clock                              0x000000c9   Thumb Code     0  entry7b.o(.ARM.Collect$$$$00000008)
    _main_cpp_init                           0x000000c9   Thumb Code     0  entry8b.o(.ARM.Collect$$$$0000000A)
    _main_init                               0x000000c9   Thumb Code     0  entry9a.o(.ARM.Collect$$$$0000000B)
    __rt_final_cpp                           0x000000d1   Thumb Code     0  entry10a.o(.ARM.Collect$$$$0000000D)
    __rt_final_exit                          0x000000d1   Thumb Code     0  entry11a.o(.ARM.Collect$$$$0000000F)
    vPortSVCHandler                          0x000000d5   Thumb Code    32  port.o(.emb_text)
    __asm___6_port_c_39a90d8d__prvStartFirstTask 0x000000f9   Thumb Code    28  port.o(.emb_text)
    xPortPendSVHandler                       0x00000119   Thumb Code    72  port.o(.emb_text)
    vPortGetIPSR                             0x00000165   Thumb Code     6  port.o(.emb_text)
    vListInitialise                          0x0000016b   Thumb Code    26  list.o(.text)
    vListInitialiseItem                      0x00000185   Thumb Code     6  list.o(.text)
    vListInsertEnd                           0x0000018b   Thumb Code    24  list.o(.text)
    vListInsert                              0x000001a3   Thumb Code    52  list.o(.text)
    uxListRemove                             0x000001d7   Thumb Code    40  list.o(.text)
    xTaskCreate                              0x0000036b   Thumb Code    96  tasks.o(.text)
    xTaskIncrementTick                       0x000003f5   Thumb Code   238  tasks.o(.text)
    xTaskResumeAll                           0x000004e3   Thumb Code   196  tasks.o(.text)
    vTaskSuspendAll                          0x00000671   Thumb Code    12  tasks.o(.text)
    vTaskDelayUntil                          0x0000067d   Thumb Code   106  tasks.o(.text)
    eTaskGetState                            0x000006e7   Thumb Code    76  tasks.o(.text)
    vTaskSwitchContext                       0x00000733   Thumb Code   100  tasks.o(.text)
    vTaskSuspend                             0x00000797   Thumb Code   160  tasks.o(.text)
    vTaskResume                              0x0000086f   Thumb Code   104  tasks.o(.text)
    xTaskResumeFromISR                       0x000008d7   Thumb Code   130  tasks.o(.text)
    vTaskStartScheduler                      0x00000967   Thumb Code    72  tasks.o(.text)
    vTaskEndScheduler                        0x000009af   Thumb Code    32  tasks.o(.text)
    xTaskGetTickCount                        0x000009cf   Thumb Code     6  tasks.o(.text)
    xTaskGetTickCountFromISR                 0x000009d5   Thumb Code     8  tasks.o(.text)
    uxTaskGetNumberOfTasks                   0x000009dd   Thumb Code     6  tasks.o(.text)
    pcTaskGetName                            0x000009e3   Thumb Code    20  tasks.o(.text)
    vTaskGetInfo                             0x00000a0d   Thumb Code   190  tasks.o(.text)
    uxTaskGetSystemState                     0x00000b35   Thumb Code   134  tasks.o(.text)
    vTaskPlaceOnEventList                    0x00000bbb   Thumb Code    28  tasks.o(.text)
    vTaskPlaceOnUnorderedEventList           0x00000bd7   Thumb Code    40  tasks.o(.text)
    xTaskRemoveFromEventList                 0x00000bff   Thumb Code   104  tasks.o(.text)
    xTaskRemoveFromUnorderedEventList        0x00000c67   Thumb Code    94  tasks.o(.text)
    vTaskSetTimeOutState                     0x00000cc5   Thumb Code    14  tasks.o(.text)
    xTaskCheckForTimeOut                     0x00000cd3   Thumb Code    84  tasks.o(.text)
    vTaskMissedYield                         0x00000d27   Thumb Code     8  tasks.o(.text)
    uxTaskGetTaskNumber                      0x00000d2f   Thumb Code    14  tasks.o(.text)
    vTaskSetTaskNumber                       0x00000d3d   Thumb Code     8  tasks.o(.text)
    uxTaskResetEventItemValue                0x00000d45   Thumb Code    24  tasks.o(.text)
    ulTaskNotifyTake                         0x00000d5d   Thumb Code   108  tasks.o(.text)
    xTaskNotifyWait                          0x00000dc9   Thumb Code   150  tasks.o(.text)
    xTaskGenericNotify                       0x00000e5f   Thumb Code   178  tasks.o(.text)
    xTaskGenericNotifyFromISR                0x00000f11   Thumb Code   282  tasks.o(.text)
    vTaskNotifyGiveFromISR                   0x0000102b   Thumb Code   154  tasks.o(.text)
    xTaskNotifyStateClear                    0x000010c5   Thumb Code    48  tasks.o(.text)
    pvPortMalloc                             0x0000110d   Thumb Code    98  heap_1.o(.text)
    vPortFree                                0x0000116f   Thumb Code     2  heap_1.o(.text)
    vPortInitialiseBlocks                    0x00001171   Thumb Code     8  heap_1.o(.text)
    xPortGetFreeHeapSize                     0x00001179   Thumb Code    12  heap_1.o(.text)
    pxPortInitialiseStack                    0x000011a7   Thumb Code    30  port.o(.text)
    vPortSetupTimerInterrupt                 0x000011c5   Thumb Code    16  port.o(.text)
    xPortStartScheduler                      0x000011d5   Thumb Code    42  port.o(.text)
    vPortEndScheduler                        0x000011ff   Thumb Code     2  port.o(.text)
    vPortEnterCritical                       0x00001201   Thumb Code    30  port.o(.text)
    vPortExitCritical                        0x0000121f   Thumb Code    28  port.o(.text)
    xPortSysTickHandler                      0x0000123b   Thumb Code    48  port.o(.text)
    vTaskFunction                            0x00001279   Thumb Code    34  main.o(.text)
    main                                     0x0000129b   Thumb Code    58  main.o(.text)
    vApplicationIdleHook                     0x000012d5   Thumb Code    12  main.o(.text)
    vPrintString                             0x000012fd   Thumb Code    20  basic_io.o(.text)
    vPrintStringAndNumber                    0x00001311   Thumb Code    26  basic_io.o(.text)
    fputc                                    0x0000132b   Thumb Code    30  basic_io.o(.text)
    Reset_Handler                            0x00001355   Thumb Code     4  startup_mps_cm3.o(.text)
    NMI_Handler                              0x00001359   Thumb Code     2  startup_mps_cm3.o(.text)
    HardFault_Handler                        0x0000135b   Thumb Code     2  startup_mps_cm3.o(.text)
    MemManage_Handler                        0x0000135d   Thumb Code     2  startup_mps_cm3.o(.text)
    BusFault_Handler                         0x0000135f   Thumb Code     2  startup_mps_cm3.o(.text)
    UsageFault_Handler                       0x00001361   Thumb Code     2  startup_mps_cm3.o(.text)
    SVC_Handler                              0x00001363   Thumb Code     2  startup_mps_cm3.o(.text)
    DebugMon_Handler                         0x00001365   Thumb Code     2  startup_mps_cm3.o(.text)
    PendSV_Handler                           0x00001367   Thumb Code     2  startup_mps_cm3.o(.text)
    SysTick_Handler                          0x00001369   Thumb Code     2  startup_mps_cm3.o(.text)
    AACI_IRQHandler                          0x0000136b   Thumb Code     0  startup_mps_cm3.o(.text)
    CAN_IRQHandler                           0x0000136b   Thumb Code     0  startup_mps_cm3.o(.text)
    CHLCD_IRQHandler                         0x0000136b   Thumb Code     0  startup_mps_cm3.o(.text)
    CLCD_IRQHandler                          0x0000136b   Thumb Code     0  startup_mps_cm3.o(.text)
    CPU_CLCD_IRQHandler                      0x0000136b   Thumb Code     0  startup_mps_cm3.o(.text)
    ENET_IRQHandler                          0x0000136b   Thumb Code     0  startup_mps_cm3.o(.text)
    FLEXRAY_IRQHandler                       0x0000136b   Thumb Code     0  startup_mps_cm3.o(.text)
    I2C_IRQHandler                           0x0000136b   Thumb Code     0  startup_mps_cm3.o(.text)
    LIN_IRQHandler                           0x0000136b   Thumb Code     0  startup_mps_cm3.o(.text)
    MCIA_IRQHandler                          0x0000136b   Thumb Code     0  startup_mps_cm3.o(.text)
    MCIB_IRQHandler                          0x0000136b   Thumb Code     0  startup_mps_cm3.o(.text)
    RTC_IRQHandler                           0x0000136b   Thumb Code     0  startup_mps_cm3.o(.text)
    SPI_IRQHandler                           0x0000136b   Thumb Code     0  startup_mps_cm3.o(.text)
    TIM0_IRQHandler                          0x0000136b   Thumb Code     0  startup_mps_cm3.o(.text)
    TIM2_IRQHandler                          0x0000136b   Thumb Code     0  startup_mps_cm3.o(.text)
    UART0_IRQHandler                         0x0000136b   Thumb Code     0  startup_mps_cm3.o(.text)
    UART1_IRQHandler                         0x0000136b   Thumb Code     0  startup_mps_cm3.o(.text)
    UART2_IRQHandler                         0x0000136b   Thumb Code     0  startup_mps_cm3.o(.text)
    UART3_IRQHandler                         0x0000136b   Thumb Code     0  startup_mps_cm3.o(.text)
    UART4_IRQHandler                         0x0000136b   Thumb Code     0  startup_mps_cm3.o(.text)
    USBDC_IRQHandler                         0x0000136b   Thumb Code     0  startup_mps_cm3.o(.text)
    USBHC_IRQHandler                         0x0000136b   Thumb Code     0  startup_mps_cm3.o(.text)
    WDT_IRQHandler                           0x0000136b   Thumb Code     0  startup_mps_cm3.o(.text)
    __aeabi_memset                           0x00001371   Thumb Code    14  memseta.o(.text)
    __aeabi_memset4                          0x00001371   Thumb Code     0  memseta.o(.text)
    __aeabi_memset8                          0x00001371   Thumb Code     0  memseta.o(.text)
    __aeabi_memclr                           0x0000137f   Thumb Code     4  memseta.o(.text)
    __aeabi_memclr4                          0x0000137f   Thumb Code     0  memseta.o(.text)
    __aeabi_memclr8                          0x0000137f   Thumb Code     0  memseta.o(.text)
    _memset$wrapper                          0x00001383   Thumb Code    18  memseta.o(.text)
    __aeabi_uidiv                            0x00001395   Thumb Code     0  uidiv.o(.text)
    __aeabi_uidivmod                         0x00001395   Thumb Code    44  uidiv.o(.text)
    __scatterload                            0x000013c1   Thumb Code    28  init.o(.text)
    __scatterload_rt2                        0x000013c1   Thumb Code     0  init.o(.text)
    __0printf$3                              0x000013e5   Thumb Code    22  printf3.o(i.__0printf$3)
    __1printf$3                              0x000013e5   Thumb Code     0  printf3.o(i.__0printf$3)
    __2printf                                0x000013e5   Thumb Code     0  printf3.o(i.__0printf$3)
    __scatterload_copy                       0x00001405   Thumb Code    14  handlers.o(i.__scatterload_copy)
    __scatterload_null                       0x00001413   Thumb Code     2  handlers.o(i.__scatterload_null)
    __scatterload_zeroinit                   0x00001415   Thumb Code    14  handlers.o(i.__scatterload_zeroinit)
    Region$$Table$$Base                      0x00001604   Number         0  anon$$obj.o(Region$$Table)
    Region$$Table$$Limit                     0x00001624   Number         0  anon$$obj.o(Region$$Table)
    pxCurrentTCB                             0x10000000   Data           4  tasks.o(.data)
    pcTextForTask1                           0x10000044   Data           4  main.o(.data)
    pcTextForTask2                           0x10000048   Data           4  main.o(.data)
    ulIdleCycleCount                         0x1000004c   Data           4  main.o(.data)
    __stdout                                 0x10000050   Data           4  stdout.o(.data)
    ulTaskNumber                             0x10001108   Data          12  main.o(.bss)
    __initial_sp                             0x10001318   Data           0  startup_mps_cm3.o(STACK)



==============================================================================

Memory Map of the image

  Image Entry point : 0x000000c1

  Load Region LR_IROM1 (Base: 0x00000000, Size: 0x00001678, Max: 0x00080000, ABSOLUTE)

    Execution Region ER_IROM1 (Exec base: 0x00000000, Load base: 0x00000000, Size: 0x00001624, Max: 0x00080000, ABSOLUTE)

    Exec Addr    Load Addr    Size         Type   Attr      Idx    E Section Name        Object

    0x00000000   0x00000000   0x000000c0   Data   RO          245    RESET               startup_mps_cm3.o
    0x000000c0   0x000000c0   0x00000000   Code   RO          250  * .ARM.Collect$$$$00000000  mc_w.l(entry.o)
    0x000000c0   0x000000c0   0x00000004   Code   RO          520    .ARM.Collect$$$$00000001  mc_w.l(entry2.o)
    0x000000c4   0x000000c4   0x00000004   Code   RO          523    .ARM.Collect$$$$00000004  mc_w.l(entry5.o)
    0x000000c8   0x000000c8   0x00000000   Code   RO          525    .ARM.Collect$$$$00000008  mc_w.l(entry7b.o)
    0x000000c8   0x000000c8   0x00000000   Code   RO          527    .ARM.Collect$$$$0000000A  mc_w.l(entry8b.o)
    0x000000c8   0x000000c8   0x00000008   Code   RO          528    .ARM.Collect$$$$0000000B  mc_w.l(entry9a.o)
    0x000000d0   0x000000d0   0x00000000   Code   RO          530    .ARM.Collect$$$$0000000D  mc_w.l(entry10a.o)
    0x000000d0   0x000000d0   0x00000000   Code   RO          532    .ARM.Collect$$$$0000000F  mc_w.l(entry11a.o)
    0x000000d0   0x000000d0   0x00000004   Code   RO          521    .ARM.Collect$$$$00002712  mc_w.l(entry2.o)
    0x000000d4   0x000000d4   0x00000096   Code   RO          167    .emb_text           port.o
    0x0000016a   0x0000016a   0x00000094   Code   RO           85    .text               list.o
    0x000001fe   0x000001fe   0x00000002   PAD
    0x00000200   0x00000200   0x00000f0c   Code   RO          115    .text               tasks.o
    0x0000110c   0x0000110c   0x00000084   Code   RO          152    .text               heap_1.o
    0x00001190   0x00001190   0x000000e8   Code   RO          168    .text               port.o
    0x00001278   0x00001278   0x00000084   Code   RO          198    .text               main.o
    0x000012fc   0x000012fc   0x00000058   Code   RO          221    .text               basic_io.o
    0x00001354   0x00001354   0x0000001c   Code   RO          246    .text               startup_mps_cm3.o
    0x00001370   0x00001370   0x00000024   Code   RO          255    .text               mc_w.l(memseta.o)
    0x00001394   0x00001394   0x0000002c   Code   RO          535    .text               mc_w.l(uidiv.o)
    0x000013c0   0x000013c0   0x00000024   Code   RO          550    .text               mc_w.l(init.o)
    0x000013e4   0x000013e4   0x00000020   Code   RO          348    i.__0printf$3       mc_w.l(printf3.o)
    0x00001404   0x00001404   0x0000000e   Code   RO          562    i.__scatterload_copy  mc_w.l(handlers.o)
    0x00001412   0x00001412   0x00000002   Code   RO          563    i.__scatterload_null  mc_w.l(handlers.o)
    0x00001414   0x00001414   0x0000000e   Code   RO          564    i.__scatterload_zeroinit  mc_w.l(handlers.o)
    0x00001422   0x00001422   0x00000002   PAD
    0x00001424   0x00001424   0x000001b8   Code   RO          355    i._printf_core      mc_w.l(printf3.o)
    0x000015dc   0x000015dc   0x00000027   Data   RO          200    .conststring        main.o
    0x00001603   0x00001603   0x00000001   PAD
    0x00001604   0x00001604   0x00000020   Data   RO          560    Region$$Table       anon$$obj.o


    Execution Region RW_IRAM1 (Exec base: 0x10000000, Load base: 0x00001624, Size: 0x00001318, Max: 0x00008000, ABSOLUTE)

    Exec Addr    Load Addr    Size         Type   Attr      Idx    E Section Name        Object

    0x10000000   0x00001624   0x00000038   Data   RW          117    .data               tasks.o
    0x10000038   0x0000165c   0x00000008   Data   RW          154    .data               heap_1.o
    0x10000040   0x00001664   0x00000004   Data   RW          169    .data               port.o
    0x10000044   0x00001668   0x0000000c   Data   RW          201    .data               main.o
    0x10000050   0x00001674   0x00000004   Data   RW          534    .data               mc_w.l(stdout.o)
    0x10000054        -       0x000000b4   Zero   RW          116    .bss                tasks.o
    0x10000108        -       0x00001000   Zero   RW          153    .bss                heap_1.o
    0x10001108        -       0x0000000c   Zero   RW          199    .bss                main.o
    0x10001114   0x00001678   0x00000004   PAD
    0x10001118        -       0x00000200   Zero   RW          243    STACK               startup_mps_cm3.o


==============================================================================

Image component sizes


      Code (inc. data)   RO Data    RW Data    ZI Data      Debug   Object Name

        88         12          0          0          0       2203   basic_io.o
         0          0          0          0          0      11696   croutine.o
         0          0          0          0          0       1452   event_groups.o
       132         12          0          8       4096       1936   heap_1.o
       148          0          0          0          0       1838   list.o
       132         28         39         12         12       1572   main.o
       382         26          0          4          0       7036   port.o
        28          4        192          0        512        760   startup_mps_cm3.o
      3852        240          0         56        180      27003   tasks.o

    ----------------------------------------------------------------------
      4764        322        264         80       4804      55496   Object Totals
         0          0         32          0          0          0   (incl. Generated)
         2          0          1          0          4          0   (incl. Padding)

    ----------------------------------------------------------------------

      Code (inc. data)   RO Data    RW Data    ZI Data      Debug   Library Member Name

         0          0          0          0          0          0   entry.o
         0          0          0          0          0          0   entry10a.o
         0          0          0          0          0          0   entry11a.o
         8          4          0          0          0          0   entry2.o
         4          0          0          0          0          0   entry5.o
         0          0          0          0          0          0   entry7b.o
         0          0          0          0          0          0   entry8b.o
         8          4          0          0          0          0   entry9a.o
        30          0          0          0          0          0   handlers.o
        36          8          0          0          0         68   init.o
        36          0          0          0          0        108   memseta.o
       472         14          0          0          0        184   printf3.o
         0          0          0          4          0          0   stdout.o
        44          0          0          0          0         80   uidiv.o

    ----------------------------------------------------------------------
       640         30          0          4          0        440   Library Totals
         2          0          0          0          0          0   (incl. Padding)

    ----------------------------------------------------------------------

      Code (inc. data)   RO Data    RW Data    ZI Data      Debug   Library Name

       638         30          0          4          0        440   mc_w.l

    ----------------------------------------------------------------------
       640         30          0          4          0        440   Library Totals

    ----------------------------------------------------------------------

==============================================================================


      Code (inc. data)   RO Data    RW Data    ZI Data      Debug   

      5404        352        264         84       4804      55308   Grand Totals
      5404        352        264         84       4804      55308   ELF Image Totals
      5404        352        264         84          0          0   ROM Totals

==============================================================================

    Total RO  Size (Code + RO Data)                 5668 (   5.54kB)
    Total RW  Size (RW Data + ZI Data)              4888 (   4.77kB)
    Total ROM Size (Code + RO Data + RW Data)       5752 (   5.62kB)

==============================================================================

